:10F80000B240805A200132C23D4000F931408002AE
:10F81000F24080005600F2400F005700C2435800EB
:10F82000F240AA002200C2432100F24080002A00D8
:10F83000F24080002900C2432E00B240D200720183
:10F84000B24010026001B2401000620182436401C4
:10F85000F2403F000002F2403F000102C2430202B8
:10F86000C243030232D25B4220007BF055007B9002
:10F87000550005247A40AA00B0128EF8F43F3D40AE
:10F8800000F9F13F6A43B0128EF8FD233041F2C017
:10F890008000290005433D40F8F835909800FD3B75
:10F8A00005433D4000F935909800FD3B364000028D
:10F8B0007746784239402E004757022C39401700CE
:10F8C0003D40F8F8054335901700FD3B3D4000F9F9
:10F8D00005430599FE3B5883ED2336900402E82347
:10F8E000054335901700FD3BF2C0AA002100F2D07D
:10F8F000800029003041004DC2EA21001553001359
:0AF90000F2C0AA0021001553001305
:10FFE80000000000000000000000F6F8000000001B
:08FFF80000000000000000F809
:00000001FF
